:030000000219FDE5
:03000B000200AA46
:03002B0002015F70
:03005B000202F5A9
:030073000202DBAB
:1000800002030406080C10182030406080040608A3
:100090000C10182030406080A0C000070F1F3F0DDB
:1000A0000D0403060D0502030202C2AFC0D0C0E07A
:1000B000206217E5256002E473E525F4F58A758B67
:1000C00000D262D0E0D0D0D2AF3285268AC262E5BB
:1000D00026F4602F758B00D0E0D0D0D297D295D285
:1000E00093D2AF32D297D295D293206E0C2066096C
:1000F000740AD5E0FDE57E4290758B00D0E0D0D04B
:10010000D2AF32758A00C28DD26201F901B930686E
:1001100005206602C29701B9306805206602C295C3
:1001200001B9306805206602C29301B9C2963068F1
:100130000A2066077408D5E0FDC29701B9C2943061
:10014000680A2066077408D5E0FDC29501B9C2921D
:1001500030680A2066077408D5E0FDC29301B9C271
:10016000AFC2AD53E6EFC0D0C0E0D2D3D2AFC2CE63
:10017000E52A6007207449152A21C07800790020FB
:10018000742EE580307E01F430E50278FF53DACF3B
:10019000207E0343DA20307E0343DA10C2D8C271D6
:1001A000E580307E01F430E50279FFC3E89970CB39
:1001B000306103752A40207403752A40885FD2702D
:1001C00020740DE52B6004152B21D043DA01C2D831
:1001D00020700221E3A85F206102C2702074022116
:1001E000E188227882B60403852224C3E525944061
:1001F0004002D26420CF0AD0E0D0D043E610D2AD86
:1002000032C2CF053A7802E52A6005307402152A19
:10021000C3E55F94014005756200412D756300756B
:100220006C00E5622401F56250037562FF7982B7C4
:10023000020D306D1DC3E52294324016854D2279A2
:1002400082B7030E306D0BC3E52294324004798EE1
:100250008722C3E5239522600840041523416105E8
:1002600023D8CA056CE56C7002156CD56D63756D8D
:10027000017805C3E56C956E4057C3E56C956F50EA
:10028000087801756D03020295C3E56C9570500501
:100290007801756D01C3E5659524401E7982B70428
:1002A0000241C6206D14852465E56C046003856EEB
:1002B0006C756D0175233C0202D1E565285005750A
:1002C00065FF41C6F565E5650470067563FF756CED
:1002D000FFD0E0D0D043E610D2AD32C2AFC0D05391
:1002E000E67FC26075910085569485579575910497
:1002F000D0D0D2AF32C2AF53E6EFC2ADC0D0C0E073
:10030000C0F0D2D3D2AFA8FBA9FCC2D83071026131
:100310005C53DACF207E0343DA10307E0343DA20C9
:10032000D271E580307E01F420E5026133882789AF
:1003300028A13B53DACF207E0343DA20307E0343EB
:10034000DA10C2D8C271307402A1277800E580307B
:100350007E01F430E502A127885FA10F53DACF2098
:100360007E0343DA20307E0343DA10C2712061023B
:10037000813553DACF207E0343DA10307E0343DA2F
:1003800020C2D8D271885A895BC3E89558F8E9959C
:1003900059F97B007E087A00C3E8948CE9940050F8
:1003A00005755E008127882178A2E6A8216055C3E3
:1003B000E894C8E994005008E4D2E4FB7A0A810288
:1003C000C3E89468E994015008E4D2E3FB7A0F8112
:1003D00002C3E894D0E994025008E4D2E2FB7A1E0A
:1003E0008102C3E894A0E994055008E4D2E1FB7AC5
:1003F0003C8102C3E89498E994085008E4D2E0FBF9
:100400007A787E00C3E8955CFCE9955DFD30E70AEB
:10041000ECF42401FCEDF43400FD755E00C3EC9AAD
:10042000ED9E5003755E01885C895D855A58855B39
:10043000597802A10FC3E89527F8E99528F9307C8F
:100440000281F3307B0281F3307A0281EC20750265
:100450008158E9FDE8FC8177E9C313F9E813F83026
:10046000790281ECE9C313F9E813F830780281ECE2
:0F047000E9C313FDE813FC206126C3EC941CEDD7
:10047F0094024002818EED7018C3EC94C85012059F
:10048F0029C3E529940A5002A127755F00D270A1F4
:10049F0027E529600215297400207F037896E6244A
:1004AF00FAFEE43400FFC3EC9EFCED9FFD5006788E
:1004BF0000790081F3C3EC94FFED9400400678FFC0
:1004CF00790081F3EC8575F0A4C5F0A2F733F879C4
:1004DF0000400302050F78FF790002050FE9C313EF
:1004EF00F9E813F8307C0EE9600278FFC3E813389F
:1004FF00F8E43400F9C3E894FFE99400400278FF70
:10050F00885FD270206102A127741FF4552F4BF51D
:10051F002FC274EB7002D274752A40307403752A9F
:10052F000A306102A13B20740353DAFE2074037575
:10053F002B20D0F0D0E0D0D0D2AD43E610327901ED
:10054F0002056B790302056B790A02056B791E02AE
:10055F00056B796402056B79C802056B7817E4D5D2
:10056F00E0FDD8FAD9F6227A147B780205927A1038
:10057F007B8C0205927A0D7BB40205927A0B7BC8B5
:10058F000205927902B27DE4C294D5E0FDC295D501
:10059F00E0FDD295D5E0FDD294D5E0FDC297E5768A
:1005AF00D5E0FDD2977496D5E0FDD9D9EAF8D5E01C
:1005BF00FDD8FBDBCEC29422C37C007D0075F0001A
:1005CF0005F0EA33FAEB33FB50F6EB13FBEA13FAC1
:1005DF00C3E9FFE8FEE89AF8E99BF95004EFF9EE5A
:1005EF00F8B3EC33FCED33FDD5F0DFEDF9ECF82289
:1005FF00E889F08A20D2D4F8A9F07B0030F70B7B82
:10060F00FFF42401F8E9F43400F9E88520F0A4ADF3
:10061F00F0F8E98520F0A4AFF0FEED2EF974003F5D
:10062F00FA7C04C3EA13FAE913F9E813F8DCF48B44
:10063F00F030F70AE8F42401F8E9F43400F9E88916
:10064F00F0C2D4F8A9F0227882B604030206F5C3EB
:10065F00E55F9419401EE52D54067018206D36780D
:10066F00057994E7146007780A1460027812C3E5DD
:10067F004198401F306D09856765756CFF756D0179
:10068F00852224E4F545F546F547F548F549C26D51
:10069F000206F5D26D7994E7147013E523F4333322
:1006AF00F913F8E9540104F9E854FE0206E9E714D6
:1006BF00147014E523F4333333F913F8E9540304B6
:1006CF00F9E854FC0206F1E523F433333333F9131D
:1006DF00F8E954070404F9E854F8C39440F8E9948E
:1006EF0000F98845894622C3E54113F9E54013F81F
:1006FF00C3E54598F8E54699F9500CC3E89480E9AD
:10070F0094FF401602072DC3E8947FE9940050032D
:10071F0002072D787F790002072D788079FF884AAC
:10072F00894B22E54A2547F8E54B3548F9854B209B
:10073F00E4300701F43549FA30E709C3EA94F04091
:10074F001502076BC3EA940F500302076B78FF790A
:10075F00FF7A0F02076B780079007AF0C3E52495D2
:10076F0064500AC374019524500B020789E54B208E
:10077F00E70E020789E54B30E706884789488A4923
:10078F002278A4E6FAC3E54A33F8E54B33F9B1FF13
:10079F00E930E70BC3E89480E994FF4013E1C3C34A
:1007AF00E8947FE994005002E1C3787F7900E1C3B8
:1007BF00788079FFE820E715C3E52398F84009C34F
:1007CF00E8940140030207EA78010207EAE8F424FB
:1007DF00012523F840030207EA78FF884C2278A509
:1007EF00E6FAA848A949B1FFE930E70CC3E894013C
:1007FF00E994FF401602081EC3E894FFE9940050E5
:10080F000302081E78FF790002081E780179FFE9BC
:10081F0020E715C3E54C98F84009C3E8940140035D
:10082F000208457801020845E8F42401254CF840F8
:10083F000302084578FF88242278FFC26420693DAF
:10084F00206A12D264C3E541940A4009C3E5259496
:10085F00405002C26479A1E76023E541601F74FF35
:0F086F008541F0848539F0306A0375F005A4F8EF
:10087E00C5F0600278FFC3E895675002A8678866E6
:10088E0022C3E5409440E5419401E566500314010E
:10089E00A0046002F566227883E6F520120F3E75FD
:1008AE00E89012054D75E890E5E820ECFBA8BDA98F
:1008BE00BE120FD8757155757200C3740013FD7496
:1008CE0055606613FC74552CFC74003DFDECFAED7E
:1008DE00FBC3E89AE99B4014E5712455F571E57266
:1008EE003400F572EA2CFAEB3DFB80E5AE71AF7287
:1008FE00C3E57213F9E57113F8C3E913F9E813F8B8
:10090E007A03C3E913F9E813F8DAF7AA201A700983
:10091E007571007572000209371AEA6008EE28FE3A
:10092E00EF39FFDAF88E718F722275E89022788394
:10093E00E6FFE5E820ECF7A8BDA9BE0573C3E57395
:10094E0094084052757300E9FA79A0E76044EA70A2
:10095E0007E574601B020972C3E895746010E574B4
:10096E005006600C1402097E0460F902097EE574DB
:10097E00F574C3946D401B7564C0C3940440137525
:10098E006480C39404400B756440C39404400375A3
:10099E00640075BB0822EFC39401601F7455601B81
:1009AE00C3E894FFE994035012C3E89571E9957278
:1009BE005009E564600C15640209D0E564F4600228
:1009CE000564A864C3E524985002A824C3E895657D
:1009DE00400AA865E565F460038565648825882668
:1009EE00E573B4070375BB1022743279A687F0A4A1
:1009FE00C5F0A2F733F8C3E895644002A8648822D4
:100A0E008824882588268867227540007541F02243
:100A1E00C2AF75C820A8CCA9CDAA3A30CF010A75AD
:100A2E00C824D2AFAB3BAC3C883B893CC3E89BF8B7
:100A3E00E99C206908F930670261334190AD3D8A27
:100A4E003DF9EA9DFA600478FF79FFAE3EAF3F8B29
:100A5E003E8C3FC3EC9FFCC3E99CF542A83BA93CEE
:100A6E00C3E89EF8E99FF9C3E54113FBE54013FA8D
:100A7E00E82AF540E93BF54150067540FF7541FF08
:100A8E0041DAAA40AB41AC40AD417E047F02C3EBDC
:100A9E00940440021E1FC3EB940840021E1FC3EDB8
:100AAE0013FDEC13FCDEF7C3EA9CFAEB9DFBEF6043
:100ABE0009C3E913F9E813F8DFF7EA28FAEB39FB73
:100ACE008A408B4150067BFF8B408B41C3EB9402D7
:100ADE005002D2673069047F0361057892E6FFC346
:100AEE00E537948240110FC3E53794A040010FC340
:100AFE00EF940640027F057E05E541C4540FF9E5EB
:100B0E0041C454F0F8E540C4540F28F8C3E89EFAE7
:100B1E00E99400FB4009C3EA9402EB940050047A76
:100B2E0002E4FB617FAA40AB41EBC4FEEAC4540F62
:100B3E004EFCC3EA9CFAEB9400FBC3E813C313F814
:100B4E00EA28FAEB3400FB8A408B41C3EB94024057
:100B5E0002C2677805EBC4FE7B00EAC4540F4EFA5E
:100B6E00C3EA98FA4005C3940250027A027892E6DC
:100B7E00FF306002617F855256855357D26043E63F
:100B8E0080C3E49AF8E49BF93067028119E8FAE928
:100B9E00FBD3E913FDE813FC88528953C3EF94038A
:100BAE006038EF20E00DE82CF8E93DF9ECFAEDFBAA
:100BBE00020BD4E828F8E939F9C3E82402F8E9343D
:100BCE0000F97AFE7BFFC3EF9403400E8A548B55D7
:100BDE00884E894F8C508D51814D885489558A4E3F
:100BEE008B4F8C508D51306920C3E53394034019DF
:100BFE00E542A2E713F8E555F4240138400B20E74F
:100C0E00087554FFF42401F555814DE8FAD3E81325
:100C1E00FC8852C3EF94036020EF20E007E82CF825
:100C2E00ECFA8139E8282402F87AFEC3EF940340E7
:100C3E00088A54884E8C50814D88548A4E8C50E5CB
:100C4E006BC3335002646BF56B30600281577534A1
:100C5E0002D26043E680E52D54066026A840A941E5
:0F0C6E00C3E913F9E813F8C2AF53E67F7591009D
:100C7D00C3E498F594E499F595759104D26043E633
:100C8D0080D2AF22D265754400752000306B03759C
:100C9D002040020CB0D265754400752040306B03C6
:100CAD00752000D2AF7801206722E52D5406600231
:100CBD00C265C3E541940540137802940540087858
:100CCD0003940540027806306902780A206019E520
:100CDD0044601530690AC3E53394034003D53406E7
:100CED00D2AFD26CA181915FD2AF0000C2AF2067AD
:100CFD0026E541C3FB940F40027B0FEB24053073B7
:100D0D000123306A02742820620123F930690279C7
:100D1D0082E58BC39940B50544E59B5440B520024F
:100D2D00A16B30690A08C3E8940A40010881D920F3
:100D3D00650281B0C26553E67F759100306710750D
:100D4D0094007595FE759104D26043E68081B0AE36
:100D5D0040AF41C3E49EF594E49FF595A152C3E5E0
:100D6D00339402500281B030650281B0D802A17F68
:100D7D0081D9C26C53E67F75910085549485559544
:100D8D00759104854E56854F57D26043E680D2AF9C
:100D9D00E52D54066008206A020533020DBB306C48
:100DAD000D206B0A2065071581158102160B22781F
:100DBD00003064053065027801E53775F007A4F958
:100DCD00E5F028F5F0E9A2F013A2F113A2F213F564
:100DDD0037C394785003753778C3E5379538400895
:100DED00D266D297D295D293306002A1F585505636
:100DFD00855157D26043E68022207D11C2AF7543E5
:100E0D0002C294D296D2AF759F10020FD5C2AF75A4
:100E1D004302C294D292D2AF759F10020FD5307299
:100E2D0043207D20C2AF75430390013D757E10D2E6
:100E3D0093C292306204C295C149D294D2AF759FCC
:100E4D0013020FD5C2AF75430390013D757E10D2CD
:100E5D0097C296306204C295C169D294D2AF759F84
:100E6D0011020FD5207D17C2AF754303900118D223
:100E7D0093306202C295D2AF759F13020FD5C2AFE8
:100E8D00754303900118D297306202C295D2AF75A7
:100E9D009F11020FD5207D11C2AF754304C296D2AA
:100EAD0092D2AF759F11020FD5C2AF754304C29296
:100EBD00D296D2AF759F13020FD5307243207D208D
:100ECD00C2AF75430590012C757E40D295C294300A
:100EDD006204C297C1E5D296D2AF759F10020FD5AD
:100EED00C2AF75430590014E757E04D295C2943004
:100EFD006204C293E105D292D2AF759F10020FD555
:100F0D00207D17C2AF75430590010ED29530620258
:100F1D00C297D2AF759F10020FD5C2AF7543059022
:100F2D000122D2953062EBC293D2AF759F10020FA2
:100F3D00D5207D11C2AF754306C292D294D2AF7542
:100F4D009F13020FD5C2AF754306C296D294D2AF8E
:100F5D00759F11020FD5307242207D20C2AF7543AF
:100F6D000190014E757E04D297C296306204C293F1
:100F7D00E181D292D2AF759F11020FD5C2AF7543E9
:100F8D000190012C757E40D293C292306204C297BB
:100F9D00E1A1D296D2AF759F13E1D5207D16C2AFD8
:100FAD00754301900122D297306202C293D2AF7580
:100FBD009F11E1D5C2AF75430190010ED2933062FE
:100FCD0002C297D2AF759F13C2662290010C757E37
:100FDD0000D297D295D293C296C294C292C2622287
:100FED00788076070876070876010876040876FF7C
:100FFD000876FF08760908760208760108760178EA
:10100D008C76010876000876B40876FF0876FF081E
:10101D0076FF0876030876FF0876010876FF0876D6
:10102D00250876D00876780876C80876040876FF05
:10103D0008760108760008767A08760A087601089F
:10104D0076010876000876FF227887E6FFC272786F
:10105D0088C27DE630E102D27DC27E7889E630E13C
:0E106D0002D27EC3EF94026008758E01D2732A
:10107B00021083758E00C273227880E61490008074
:10108B009378A4F67881E6149000809378A5F6788F
:10109B0086E61490008D9378A6F6789FE6F870019B
:1010AB0008C3E8941140027811E82828F56E256EE4
:1010BB00256E28F56F256E2828F570789CE6753817
:1010CB00FF75390CB402067538A075390AB40306DE
:1010DB0075388275390578A3E61490009A93F569F3
:1010EB00120FD822227896E6FA7897E6FB7888E6F4
:1010FB00B40305C3EB940EFB307F047A007BFFC374
:10110B00EB9AFCC3948250027C827575000575ECDA
:10111B008575F0A4C3E5F0947D40F222D27F11F0E7
:10112B0012055C7A007B007C10120552E55F2AFAEF
:10113B0074003BFBDCF37C04C3EB13FBEA13FADC1C
:10114B00F7FEC27F11F022E5EF20E60375200005C4
:10115B0020903FFFE520146006901DFF1460009364
:10116B0004600375EF1253D9BF7581C043FF801222
:10117B00054D75EF0243B203E5B3240420E70DF5EB
:10118B0021E5E320E0068521B343E301120FD87577
:10119B0080FF75A40075F1B275D4DF7590A975A5A4
:1011AB00FC75F2FC75D50175A60175E241E4F8F604
:1011BB00D8FD756B01120FED121653789886767564
:1011CB003001C2AF12056612057612055C12057D61
:1011DB0012055C12058412055C1217761205661255
:1011EB000566120561C2AF78FA79FA308507D9FB2B
:1011FB00D8F7021C001156118411EF11F078988664
:10120B0076120FD875885075891275C8247591049C
:10121B0075D84075A82275B80275E690759B8075D8
:10122B009D0075D10E75BC5875BB0875BA1175E864
:10123B008012054DD2AF1208A553DACF207E03439F
:10124B00DA20307E0343DA1043DA01C2D8C27112BE
:10125B000566D2617B037A0CE55E70077A0CDB03C3
:10126B000211F012055C2070030211F0C270E55FF1
:10127B00C3940240E1E52F541F856160F561B560B1
:10128B00D5DAD5C26153DACF207E0343DA20307E24
:10129B000343DA10C2D8C27178A2E67008D274E5A3
:1012AB002F54E0F52FC275752900120561307409B2
:1012BB00C3E529940A4002D27512055278023074A4
:1012CB00027800C3E55F9840F0C2AF1205761205B5
:1012DB0076120576D2AF120566754D00120552785F
:1012EB008CE6C3940150030213BDE530C394015047
:1012FB00030213BD207435C3E55F94FF5003021343
:10130B00BDC2AF12058BD2AF120561C3E55F94016D
:10131B0050EFC2AF120576120557120576D2AF12F7
:10132B000561C3E55F94FF40E90217FB7F05D27FA0
:10133B0011F0120561C2AFC27F11F0AE5FC3E55F62
:10134B00947FD2AF407612054DC2AF12058BD2AF50
:10135B00DFDC3127C3EE94057897F612056612167B
:10136B009512177E7F0AD27F11F0120561C2AFC2B0
:10137B007F11F0AE5FC3E55F947FD2AF50E61205ED
:10138B004DC2AF120576120557120576D2AFDFD6D6
:10139B003127EE24057896F612056612169512176C
:1013AB00AD12056111F0C3E55F94FF500241FF02DE
:1013BB0017FBC3E55F954D4003855F4D12056178C3
:1013CB00017988E7B403027805C3E55F98400241D1
:1013DB00E7C2AF12058B12058B12058BD2AF12052C
:1013EB0066753000E4F531F5320531E531F47039CD
:1013FB000532789AE67819146012783214600D78F9
:10140B007D14600878FA146003753200C3E53298D6
:10141B00401715327531B478998676C2AF12058BA9
:10142B00D2AF78988676120561120557E52A7005BA
:10143B0030740221F078012074027806C3E55F98BE
:10144B0040A7120561E52A70030211F0C2AF120F1B
:10145B00D8E4F522F523F524F525F526F56AD2AF68
:0E146B007885E6C333F568E4F545F546F547A8
:10147900F548F549F573F52CF52DF53775730875AC
:10148900BB1012054D120938E5E820ECFBA8BDA9EF
:10149900BEE97001F8887412093C75730875BB10B0
:1014A9007887E6FE760211567887EEF6C2AF756444
:1014B900FF1209F7852264852265852266D2AF75F8
:1014C900220175240175250175260185636C756DE9
:1014D900017888E6B40307C27D307602D27DD268EE
:1014E900D269753300120F3E120F63120A17120ADE
:1014F9001E120A17120A1E120A17021512C2AF117A
:1015090056D2AF75730075BB08120CA2120656129B
:101519000DBC120E06120A1E120C91306D03120632
:10152900F620670312084830670312088F120DBCB2
:10153900120E2B120A1E120CA2306D031207321260
:101549000DBC120EA2120A1E120C91306D03120765
:1015590090120DBC120EC7120A1E120CA2306D0396
:101569001207ED120DBC120F3E120A1E1209381293
:101579000C91120DBC120F6312093C120A1E30693C
:101589002F206B2C85676485676585636C756D0194
:1015990079187A0CC3E533994009C269D26A8A3548
:1015A9000215B9C3E55F940140030215120216132F
:1015B900306A1B206B18E535147004C26AA106F560
:1015C90035C3E55F940140030215120216137536FF
:1015D90000C3E5629401400985676585636C756D93
:1015E90001C3E56278FA985021307404E52A601A3B
:1015F90078F0306B058567647820C3E5419850021F
:10160900A1120536E55F6002C116753600C2AF1238
:101619000FD87887E6FE760211567887EEF6E4F55C
:1016290022F523F524F525F526F568C268D2AF120F
:10163900054D120FD8307406E52A700221F0788D15
:10164900E6C39401400241C461EF901A0D7820125B
:1016590016D7E520B4A50CA31216D7E520B45A0372
:10166900021675120FED121695021694901A037848
:10167900807B0A1216D7A308DBF9901A0F788C7BA6
:10168900181216D7A308DBF9901A2722C2AF12172E
:10169900161216F0901A00740E1216DCA3740412B6
:1016A90016DCA374141216DC901A0378807B0A12D4
:1016B90016DBA308DBF9901A0F788C7B181216DB5E
:1016C900A308DBF9121729121707901A2722E493A6
:1016D900F622E6438F01538FFD75EF0275B7A575A5
:1016E900B7F1F0538FFE22438F02438F0175EF024A
:1016F90075B7A575B7F1901A0DF0538FFC22901AA2
:101709000D74A5D1DC901A0E745AD1DC227A307985
:10171900D07820901A40D1D7E520F709A3DAF7222B
:101729007A3079D0901A40E7D1DC09A3DAF922ABF3
:1017390077A878BB01027980BB02027981BB0302D9
:101749007982BB04027994BB05027983BB060279CD
:1017590086BB07027992BB08027987BB0902799C8B
:10176900BB0A027988BB0B027989E8F7227C05124A
:101779000566DCFB22C2AF12057612057D120584CF
:1017890012058B12055712057612057D1205841272
:10179900058B12055712057612057D12058412056F
:1017A9008BD2AF22C2AF12058B12058412057D12AE
:1017B900057612055712058B12058412057D12054F
:1017C9007612055712058B12058412057D120576CE
:1017D900D2AF22AE77AF78C2AF1205761205761274
:1017E9000576120557DEF212058B120557DFF8D27E
:1017F900AF22F17EF176121776757701757801754A
:1018090079001217DC7C05AD5F120566C3ED955FA3
:1018190070F5C3E55F9401400AC3E55F94FF403763
:1018290002183D12173812169512177EC2AF75EFBE
:1018390012121776DCD10579C3E579940350028039
:10184900C11217760578E5771490009F93F808C3BD
:10185900E57898500280A81217761217760577C393
:0E186900E577940C50028094120FED12169544
:08187700C2AF75EF12121776E3
:0319FD0002115282
:101A00000E041407070104FFFF09020101A55A0192
:101A100000B4FFFFFF03FF01FF25D078C804FF01DA
:081A200000FF0A010100FFFFB5
:101A400023536B79494949333041232020202020FA
:101A500023424C48454C4923463333302320202031
:101A60002020202020202020202020202020202076
:101C0000C2AFC2D353D9BF7581C043B20343FF8073
:101C1000752438752503B1C975EF0275E24043F1AB
:101C20002053A4DF75D400D2857DFA780379E67C51
:101C300010752200752300901DD67B0675249875BB
:101C400025013085028142208508D8FBD9F9DCF7CF
:101C500081B4308508D8FBD9F9DCF781B4B189E4C7
:101C600093A3C39A6004DDC381B4DBDBB17B600264
:101C7000812B7B08E493FAA3B15CDBF87A30B15C8A
:101C8000752200752300B17BEAFCEBFDC3ED94FEE9
:101C9000400EB17B8A278B28ED30E0048A828B834B
:101CA000B17B7AC270D8C3ED94FE601350CEBD00F4
:101CB00025EC60097520007521FF0200008100A855
:101CC00027A9280809D804D90281D3B17FEA89AAB3
:101CD000F281C50D81A0C3ED94035049EDA2E092BD
:101CE000007AC5C3E5829400E583941C50902000DF
:101CF00010438F02438F0175B7A575B7F1F030001F
:101D00001FA827A9280809438F01538FFDD804D99C
:101D100002A12089AAE275B7A575B7F1F0A3A10DBC
:101D2000538FFC817C7AC1BD030CE493A3FAB140CC
:101D3000DCF8B138817C817EAA22AB23B15CEBFA5E
:101D4000EA6222752608C3E52313F523E52213F57D
:101D50002250066323A0632201D526EAB1C9B1C986
:101D600075260AEAF4200102D285300102C285B14B
:101D7000C9C3134002C201D526EB22B17FEAFB2082
:101D80008502A17F308502A184752608AE24AF2587
:101D9000C3EF13FFEE13FEB1CDB1C9C3EA13308513
:101DA000024480FA30E703632201C3E52313F523DD
:101DB000E52213F52250066323A0632201D526D91C
:101DC000E52265236523F52222AE24AF250E0FDE22
:101DD000FEDFFCD20122424C48656C693437316326
:041DE000F3300601D5
:00000001FF
